******************************************************************************
               TMS320C6x Linker PC v7.2.1                      
******************************************************************************
>> Linked Mon Oct 17 09:56:38 2011

OUTPUT FILE NAME:   <DSP_sysbios_Static_example.out>
ENTRY POINT SYMBOL: "_c_int00"  address: 80003d40


MEMORY CONFIGURATION

         name            origin    length      used     unused   attr    fill
----------------------  --------  ---------  --------  --------  ----  --------
  IRAM                  10800000   00040000  00000000  00040000  RW X
  OCMC_0                40300000   00020000  00000000  00020000  RW X
  OCMC_1                40400000   00020000  00000000  00020000  RW X
  DDR3_RAM              80000000   10000000  0000db12  0fff24ee  RWIX


SECTION ALLOCATION MAP

 output                                  attributes/
section   page    origin      length       input sections
--------  ----  ----------  ----------   ----------------
.pinit     0    80000000    00000000     UNINITIALIZED

.data      0    80000000    00000000     UNINITIALIZED

xdc.meta   0    80000000    000000e7     COPY SECTION
                  80000000    000000e7     static.p674.obj (xdc.meta)

.text      0    80000000    00008040     
                  80000000    00000ae0     static.p674.obj (.text:_xdc_runtime_System_doPrint__I)
                  80000ae0    000008e0     static.p674.obj (.text:_ti_sysbios_family_c64p_Exception_handler__I)
                  800013c0    000003e0     static.p674.obj (.text:_ti_sysbios_knl_Semaphore_pend__E)
                  800017a0    00000360     static.p674.obj (.text:_ti_sysbios_BIOS_startFunc__I)
                  80001b00    000002e0     static.p674.obj (.text:_ti_sysbios_heaps_HeapBuf_Instance_init__F)
                  80001de0    000002a0     static.p674.obj (.text:_xdc_runtime_System_printfExtend__I)
                  80002080    00000280     static.p674.obj (.text:_ti_sysbios_knl_Task_Module_startup__E)
                  80002300    00000280     static.p674.obj (.text:_xdc_runtime_Core_createObject__I)
                  80002580    00000280     static.p674.obj (.text:_xdc_runtime_Text_putSite__F)
                  80002800    00000260     rts6740.lib : imath64.obj (.text:__divull)
                  80002a60    00000260     static.p674.obj (.text:_ti_sysbios_family_c64p_Cache_Module_startup__E)
                  80002cc0    00000220     static.p674.obj (.text:_ti_sysbios_timers_dmtimer_Timer_setPeriodMicroSecs__E)
                  80002ee0    00000200     ti.sysbios.family.c64p.a674 : Hwi_disp_always.o674 (.text:_ti_sysbios_family_c64p_Hwi_dispatchAlways)
                  800030e0    00000200     static.p674.obj (.text:_ti_sysbios_knl_Swi_schedule__I)
                  800032e0    00000200     static.p674.obj (.text:_xdc_runtime_Error_raiseX__F)
                  800034e0    000001e0     static.p674.obj (.text:_deviceConfig$13)
                  800036c0    000001c0     static.p674.obj (.text:_ti_sysbios_knl_Task_checkStacks__E)
                  80003880    000001c0     static.p674.obj (.text:_xdc_runtime_Startup_startMods__I)
                  80003a40    00000180     static.p674.obj (.text:_xdc_runtime_LoggerBuf_Object__create__S)
                  80003bc0    00000180     ti.sysbios.family.c64p.a674 : Exception_asm.o674 (.text)
                  80003d40    00000160     static.p674.obj (.text:_c_int00)
                  80003ea0    00000160     static.p674.obj (.text:_ti_sysbios_family_c64p_Hwi_dispatchC__I)
                  80004000    00000160     static.p674.obj (.text:_ti_sysbios_knl_Clock_Object__create__S)
                  80004160    00000160     static.p674.obj (.text:_ti_sysbios_knl_Event_post__E)
                  800042c0    00000160     static.p674.obj (.text:_ti_sysbios_knl_Task_exit__E)
                  80004420    00000160     static.p674.obj (.text:_ti_sysbios_knl_Task_schedule__I)
                  80004580    00000160     static.obj (.text)
                  800046e0    00000140     static.p674.obj (.text:_ti_sysbios_family_c64p_Hwi_Module_startup__E)
                  80004820    00000140     static.p674.obj (.text:_ti_sysbios_knl_Semaphore_post__E)
                  80004960    00000140     static.p674.obj (.text:_xdc_runtime_LoggerBuf_setFilterLevel__F)
                  80004aa0    00000120     rts6740.lib : imath64.obj (.text:__divlli)
                  80004bc0    00000120     static.p674.obj (.text:_initDevice$13)
                  80004ce0    00000120     static.p674.obj (.text:_ti_sysbios_knl_Clock_workFunc__E)
                  80004e00    00000120     static.p674.obj (.text:_ti_sysbios_knl_Semaphore_Object__create__S)
                  80004f20    00000120     static.p674.obj (.text:_ti_sysbios_knl_Swi_restoreHwi__E)
                  80005040    00000120     static.p674.obj (.text:_ti_sysbios_knl_Task_startup__E)
                  80005160    00000120     static.p674.obj (.text:_xdc_runtime_LoggerBuf_getFilterLevel__F)
                  80005280    00000120     static.p674.obj (.text:_xdc_runtime_LoggerBuf_write8__F)
                  800053a0    00000120     static.p674.obj (.text:_xdc_runtime_SysMin_flush__F)
                  800054c0    00000100     rts6740.lib : sinit.obj (.text:_call_dtors)
                  800055c0    00000100     static.p674.obj (.text:_ti_sysbios_heaps_HeapBuf_Object__create__S)
                  800056c0    00000100     static.p674.obj (.text:_xdc_runtime_Memory_alloc__F)
                  800057c0    00000100     static.p674.obj (.text:_xdc_runtime_Text_putMod__F)
                  800058c0    000000e0     rts6740.lib : exit.obj (.text:_exit)
                  800059a0    000000e0                 : memset.obj (.text:_memset)
                  80005a80    000000e0     static.p674.obj (.text:_ti_sysbios_gates_GateMutex_enter__E)
                  80005b60    000000e0     static.p674.obj (.text:_ti_sysbios_knl_Mailbox_Module_startup__E)
                  80005c40    000000e0     static.p674.obj (.text:_xdc_runtime_Core_deleteObject__I)
                  80005d20    000000e0     static.p674.obj (.text:_xdc_runtime_Text_visitRope2__I)
                  80005e00    000000c0     rts6740.lib : trgdrv.obj (.text:_HOSTwrite)
                  80005ec0    000000c0                 : divu.obj (.text:__divu)
                  80005f80    000000c0                 : atexit.obj (.text:_atexit)
                  80006040    000000c0     static.p674.obj (.text:_ti_sysbios_gates_GateMutex_Object__create__S)
                  80006100    000000c0     static.p674.obj (.text:_ti_sysbios_heaps_HeapBuf_Module_startup__E)
                  800061c0    000000c0     static.p674.obj (.text:_ti_sysbios_heaps_HeapBuf_alloc__E)
                  80006280    000000c0     static.p674.obj (.text:_ti_sysbios_heaps_HeapBuf_free__E)
                  80006340    000000c0     static.p674.obj (.text:_ti_sysbios_knl_Swi_run__I)
                  80006400    000000c0     static.p674.obj (.text:_ti_sysbios_timers_dmtimer_Timer_Module_startup__E)
                  800064c0    000000c0     static.p674.obj (.text:_ti_sysbios_timers_dmtimer_Timer_stop__E)
                  80006580    000000a0     rts6740.lib : remu.obj (.text:__remu)
                  80006620    000000a0                 : memcpy64.obj (.text:_memcpy)
                  800066c0    000000a0     static.p674.obj (.text:_ti_sysbios_BIOS_exitFunc__I)
                  80006760    000000a0     static.p674.obj (.text:_ti_sysbios_knl_Clock_Instance_finalize__F)
                  80006800    000000a0     static.p674.obj (.text:_xdc_runtime_LoggerBuf_write4__F)
                  800068a0    000000a0     static.p674.obj (.text:_xdc_runtime_System_abort__F)
                  80006940    000000a0     static.p674.obj (.text:_xdc_runtime_Text_xprintf__I)
                  800069e0    00000080     rts6740.lib : llshift.obj (.text:__llshl)
                  80006a60    00000080                 : trgmsg.obj (.text:_readmsg)
                  80006ae0    00000080     static.p674.obj (.text:_ti_sysbios_BIOS_exit__E)
                  80006b60    00000080     ti.sysbios.family.c62.a674 : TaskSupport_asm.o674 (.text:_ti_sysbios_family_c62_TaskSupport_swap__E)
                  80006be0    00000080     static.p674.obj (.text:_ti_sysbios_knl_Semaphore_pendTimeout__I)
                  80006c60    00000080     static.p674.obj (.text:_ti_sysbios_knl_Swi_post__E)
                  80006ce0    00000080     static.p674.obj (.text:_ti_sysbios_knl_Task_unblockI__E)
                  80006d60    00000080     static.p674.obj (.text:_xdc_runtime_Assert_raise__I)
                  80006de0    00000080     static.p674.obj (.text:_xdc_runtime_System_rtsExit__I)
                  80006e60    00000080     static.p674.obj (.text:_xdc_runtime_Text_printVisFxn__I)
                  80006ee0    00000080     static.p674.obj (.text:ti_sysbios_hal_Hwi_checkStack:_ti_sysbios_hal_Hwi_checkStack)
                  80006f60    00000060     rts6740.lib : imath64.obj (.text:__subcull)
                  80006fc0    00000060     static.p674.obj (.text:_rtsLock$23)
                  80007020    00000060     static.p674.obj (.text:_ti_sysbios_family_c64p_Exception_Module_startup__E)
                  80007080    00000060     static.p674.obj (.text:_ti_sysbios_gates_GateHwi_Object__create__S)
                  800070e0    00000060     static.p674.obj (.text:_ti_sysbios_gates_GateMutex_Object__delete__S)
                  80007140    00000060     static.p674.obj (.text:_ti_sysbios_heaps_HeapBuf_Object__delete__S)
                  800071a0    00000060     static.p674.obj (.text:_ti_sysbios_heaps_HeapBuf_getStats__E)
                  80007200    00000060     static.p674.obj (.text:_ti_sysbios_knl_Clock_doTick__I)
                  80007260    00000060     static.p674.obj (.text:_ti_sysbios_knl_Idle_run__E)
                  800072c0    00000060     static.p674.obj (.text:_ti_sysbios_knl_Queue_Object__create__S)
                  80007320    00000060     static.p674.obj (.text:_ti_sysbios_knl_Semaphore_Instance_finalize__F)
                  80007380    00000060     static.p674.obj (.text:_ti_sysbios_knl_Task_allBlockedFunction__I)
                  800073e0    00000060     static.p674.obj (.text:_ti_sysbios_knl_Task_enter__I)
                  80007440    00000060     rts6740.lib : trgmsg.obj (.text:_writemsg)
                  800074a0    00000060     static.p674.obj (.text:_xdc_runtime_LoggerBuf_Module_startup__E)
                  80007500    00000060     static.p674.obj (.text:_xdc_runtime_LoggerBuf_Object__delete__S)
                  80007560    00000060     static.p674.obj (.text:_xdc_runtime_SysMin_putch__F)
                  800075c0    00000060     static.p674.obj (.text:ti_sysbios_hal_Hwi_initStack:_ti_sysbios_hal_Hwi_initStack)
                  80007620    00000040     rts6740.lib : sinit.obj (.text:___add_dtor)
                  80007660    00000040                 : args_main.obj (.text:__args_main)
                  800076a0    00000040                 : llshift.obj (.text:__llshru)
                  800076e0    00000040                 : abs.obj (.text:_llabs)
                  80007720    00000040     static.p674.obj (.text:_rtsUnlock$23)
                  80007760    00000040     ti.sysbios.family.c62.a674 : TaskSupport_asm.o674 (.text:_ti_sysbios_family_c62_TaskSupport_buildTaskStack)
                  800077a0    00000040     ti.sysbios.family.c64p.a674 : Hwi_asm_switch.o674 (.text:_ti_sysbios_family_xxx_Hwi_switchToIsrStack)
                  800077e0    00000040     static.p674.obj (.text:_ti_sysbios_gates_GateHwi_Handle__label__S)
                  80007820    00000040     static.p674.obj (.text:_ti_sysbios_gates_GateHwi_Object__delete__S)
                  80007860    00000040     static.p674.obj (.text:_ti_sysbios_gates_GateMutex_Handle__label__S)
                  800078a0    00000040     static.p674.obj (.text:_ti_sysbios_gates_GateMutex_Instance_finalize__F)
                  800078e0    00000040     static.p674.obj (.text:_ti_sysbios_hal_Hwi_Module_startup__E)
                  80007920    00000040     static.p674.obj (.text:_ti_sysbios_hal_Timer_Module_startup__E)
                  80007960    00000040     static.p674.obj (.text:_ti_sysbios_heaps_HeapBuf_Handle__label__S)
                  800079a0    00000040     static.p674.obj (.text:_ti_sysbios_heaps_HeapBuf_Instance_finalize__F)
                  800079e0    00000040     static.p674.obj (.text:_ti_sysbios_knl_Clock_Module_startup__E)
                  80007a20    00000040     static.p674.obj (.text:_ti_sysbios_knl_Clock_start__E)
                  80007a60    00000040     static.p674.obj (.text:_ti_sysbios_knl_Idle_loop__E)
                  80007aa0    00000040     static.p674.obj (.text:_ti_sysbios_timers_dmtimer_Timer_stub__E)
                  80007ae0    00000040     static.p674.obj (.text:_xdc_runtime_LoggerBuf_Handle__label__S)
                  80007b20    00000040     static.p674.obj (.text:_xdc_runtime_LoggerBuf_Instance_finalize__F)
                  80007b60    00000040     static.p674.obj (.text:_xdc_runtime_LoggerBuf_write0__E)
                  80007ba0    00000040     static.p674.obj (.text:_xdc_runtime_LoggerBuf_write1__E)
                  80007be0    00000040     static.p674.obj (.text:_xdc_runtime_Memory_free__E)
                  80007c20    00000040     static.p674.obj (.text:_xdc_runtime_SysMin_Module_startup__E)
                  80007c60    00000040     static.p674.obj (.text:_xdc_runtime_System_aprintf__E)
                  80007ca0    00000040     static.p674.obj (.text:_xdc_runtime_System_printf__E)
                  80007ce0    00000020     static.p674.obj (.text:___xdc__init)
                  80007d00    00000020     rts6740.lib : negll.obj (.text:__negll)
                  80007d20    00000020                 : _lock.obj (.text:__nop)
                  80007d40    00000020                 : _lock.obj (.text:__register_lock)
                  80007d60    00000020                 : _lock.obj (.text:__register_unlock)
                  80007d80    00000020                 : exit.obj (.text:_abort)
                  80007da0    00000020     static.p674.obj (.text:_nullFunc$23)
                  80007dc0    00000020     static.p674.obj (.text:_ti_sysbios_BIOS_start__E)
                  80007de0    00000020     ti.sysbios.family.c62.a674 : TaskSupport_asm.o674 (.text:_ti_sysbios_family_c62_TaskSupport_glue)
                  80007e00    00000020     static.p674.obj (.text:_ti_sysbios_family_c64p_Cache_setMar__E)
                  80007e20    00000020     static.p674.obj (.text:_ti_sysbios_family_c64p_TimestampProvider_Module_startup__E)
                  80007e40    00000020     static.p674.obj (.text:_ti_sysbios_family_c64p_ti81xx_TimerSupport_Module_startup__E)
                  80007e60    00000020     ti.sysbios.family.c64p.a674 : Hwi_asm_switch.o674 (.text:_ti_sysbios_family_xxx_Hwi_switchToTaskStack)
                  80007e80    00000020     static.p674.obj (.text:_ti_sysbios_gates_GateHwi_enter__E)
                  80007ea0    00000020     static.p674.obj (.text:_ti_sysbios_gates_GateHwi_leave__E)
                  80007ec0    00000020     static.p674.obj (.text:_ti_sysbios_gates_GateHwi_query__E)
                  80007ee0    00000020     static.p674.obj (.text:_ti_sysbios_gates_GateMutex_leave__E)
                  80007f00    00000020     static.p674.obj (.text:_ti_sysbios_gates_GateMutex_query__E)
                  80007f20    00000020     static.p674.obj (.text:_ti_sysbios_heaps_HeapBuf_isBlocking__E)
                  80007f40    00000020     static.p674.obj (.text:_ti_sysbios_knl_Swi_Module_startup__E)
                  80007f60    00000020     static.p674.obj (.text:_xdc_runtime_LoggerBuf_disable__E)
                  80007f80    00000020     static.p674.obj (.text:_xdc_runtime_LoggerBuf_enable__E)
                  80007fa0    00000020     static.p674.obj (.text:_xdc_runtime_LoggerBuf_write2__E)
                  80007fc0    00000020     static.p674.obj (.text:_xdc_runtime_Startup_exec__I)
                  80007fe0    00000020     static.p674.obj (.text:_xdc_runtime_System_Module_startup__E)
                  80008000    00000020     static.p674.obj (.text:_xdc_runtime_System_exit__F)
                  80008020    00000020     static.p674.obj (.text:_xdc_runtime_Text_visitRope__I)

.const     0    80008040    00001a74     
                  80008040    000010eb     static.p674.obj (.const:xdc_runtime_Text_charTab__A)
                  8000912b    00000001     --HOLE-- [fill = 0]
                  8000912c    000004e3     static.p674.obj (.const:.string)
                  8000960f    00000001     --HOLE-- [fill = 0]
                  80009610    000000cc     static.p674.obj (.const:xdc_runtime_Text_nodeTab__A)
                  800096dc    000000ac     static.obj (.const:.string)
                  80009788    00000040     static.p674.obj (.const:xdc_runtime_Startup_sfxnTab__A)
                  800097c8    0000003c     static.p674.obj (.const:xdc_runtime_LoggerBuf_Module__FXNS__C)
                  80009804    0000002c     static.p674.obj (.const:ti_sysbios_heaps_HeapBuf_Object__PARAMS__C)
                  80009830    00000028     static.p674.obj (.const:ti_sysbios_heaps_HeapBuf_Module__FXNS__C)
                  80009858    00000028     static.p674.obj (.const:xdc_runtime_LoggerBuf_Object__PARAMS__C)
                  80009880    00000024     static.p674.obj (.const:ti_sysbios_gates_GateHwi_Module__FXNS__C)
                  800098a4    00000024     static.p674.obj (.const:ti_sysbios_gates_GateMutex_Module__FXNS__C)
                  800098c8    00000024     static.p674.obj (.const:ti_sysbios_knl_Clock_Object__PARAMS__C)
                  800098ec    00000024     static.p674.obj (.const:ti_sysbios_knl_Semaphore_Object__PARAMS__C)
                  80009910    00000020     static.p674.obj (.const:ti_sysbios_gates_GateHwi_Object__DESC__C)
                  80009930    00000020     static.p674.obj (.const:ti_sysbios_gates_GateMutex_Object__DESC__C)
                  80009950    00000020     static.p674.obj (.const:ti_sysbios_heaps_HeapBuf_Object__DESC__C)
                  80009970    00000020     static.p674.obj (.const:ti_sysbios_knl_Clock_Object__DESC__C)
                  80009990    00000020     static.p674.obj (.const:ti_sysbios_knl_Queue_Object__DESC__C)
                  800099b0    00000020     static.p674.obj (.const:ti_sysbios_knl_Semaphore_Object__DESC__C)
                  800099d0    00000020     static.p674.obj (.const:xdc_runtime_LoggerBuf_Object__DESC__C)
                  800099f0    00000020     static.p674.obj (.const:xdc_runtime_Startup_sfxnRts__A)
                  80009a10    00000018     static.p674.obj (.const:ti_sysbios_gates_GateHwi_Object__PARAMS__C)
                  80009a28    00000018     static.p674.obj (.const:ti_sysbios_gates_GateMutex_Object__PARAMS__C)
                  80009a40    00000018     static.p674.obj (.const:ti_sysbios_knl_Queue_Object__PARAMS__C)
                  80009a58    00000018     static.p674.obj (.const:ti_sysbios_knl_Task_hooks__A)
                  80009a70    00000011     static.p674.obj (.const:_digtohex$33)
                  80009a81    00000003     --HOLE-- [fill = 0]
                  80009a84    0000000c     static.p674.obj (.const:ti_sysbios_family_c64p_Cache_initSize__C)
                  80009a90    00000008     static.p674.obj (.const:ti_sysbios_knl_Idle_funcList__A)
                  80009a98    00000004     static.p674.obj (.const:xdc_runtime_IFilterLogger_Interface__BASE__C)
                  80009a9c    00000004     static.p674.obj (.const:xdc_runtime_IGateProvider_Interface__BASE__C)
                  80009aa0    00000004     static.p674.obj (.const:xdc_runtime_IHeap_Interface__BASE__C)
                  80009aa4    00000004     static.p674.obj (.const:xdc_runtime_ILogger_Interface__BASE__C)
                  80009aa8    00000004     static.p674.obj (.const:xdc_runtime_IModule_Interface__BASE__C)
                  80009aac    00000004     --HOLE-- [fill = 0]
                  80009ab0    00000004     static.p674.obj (.const:xdc_runtime_Startup_firstFxns__A)

.far       0    80009ab8    000012f8     UNINITIALIZED
                  80009ab8    00001088     static.p674.obj (.far)
                  8000ab40    00000188     rts6740.lib : atexit.obj (.far)
                  8000acc8    000000d0                 : trgdrv.obj (.far)
                  8000ad98    0000000c                 : exit.obj (.far)
                  8000ada4    00000008                 : _lock.obj (.far)
                  8000adac    00000004                 : sinit.obj (.far)

.taskStackSection 
*          0    8000adb0    00001000     UNINITIALIZED
                  8000adb0    00001000     static.p674.obj (.taskStackSection)

.stack     0    8000bdb0    00001000     UNINITIALIZED
                  8000bdb0    00000008     static.p674.obj (.stack)
                  8000bdb8    00000ff8     --HOLE--

.cinit     0    8000cdb0    00000a0c     
                  8000cdb0    00000974     static.p674.obj (.cinit)
                  8000d724    00000004     --HOLE-- [fill = 0]
                  8000d728    0000002c     rts6740.lib : exit.obj (.cinit)
                  8000d754    00000004     --HOLE-- [fill = 0]
                  8000d758    0000001c                 : _lock.obj (.cinit)
                  8000d774    00000004     --HOLE-- [fill = 0]
                  8000d778    0000001c                 : atexit.obj (.cinit)
                  8000d794    00000004     --HOLE-- [fill = 0]
                  8000d798    0000000c                 : sinit.obj (.cinit)
                  8000d7a4    00000004     --HOLE-- [fill = 0]
                  8000d7a8    0000000a     static.obj (.cinit)
                  8000d7b2    00000006     --HOLE-- [fill = 0]
                  8000d7b8    00000004     (.pad.cinit) [fill = 0]

.bss       0    8000d7bc    00000032     UNINITIALIZED
                  8000d7bc    00000030     static.p674.obj (.bss)
                  8000d7ec    00000002     static.obj (.bss)

.args      0    8000d7f0    00000008     
                  8000d7f0    00000008     --HOLE-- [fill = 0]

.vecs      0    8000d800    00000200     
                  8000d800    00000200     static.p674.obj (.vecs)

.cio       0    8000da00    00000120     UNINITIALIZED
                  8000da00    00000120     rts6740.lib : trgmsg.obj (.cio)


GLOBAL SYMBOLS: SORTED ALPHABETICALLY BY Name 

address    name
--------   ----
8000d7bc   $bss
8000d7bc   .bss
ffffffff   .data
ffffffff   .text
80007d80   C$$EXIT
80007498   C$$IO$$
80005e00   _HOSTwrite
8000a8f8   _TSK_idle
8000da00   __CIOBUF_
8000cdb0   __STACK_END
00001000   __STACK_SIZE
00000001   __TI_args_main
80000000   ___ASM__
80000060   ___ISA__
80000078   ___PLAT__
800000a0   ___TARG__
8000ada0   ___TI_enable_exit_profile_output
ffffffff   ___TI_pprof_out_hndl
ffffffff   ___TI_prof_data_size
ffffffff   ___TI_prof_data_start
800000c0   ___TRDR__
80007620   ___add_dtor
8000ab40   ___atexit_func_id__
ffffffff   ___binit__
8000d7bc   ___bss__
8000d7f0   ___c_args__
8000cdb0   ___cinit__
ffffffff   ___data__
ffffffff   ___edata__
8000d7ee   ___end__
ffffffff   ___etext__
ffffffff   ___pinit__
ffffffff   ___text__
80007ce0   ___xdc__init
8000ab3c   ___xdc__init__addr
80007660   __args_main
80005ec0   __c6xabi_divu
80006580   __c6xabi_remu
8000ad98   __cleanup_ptr
80004aa0   __divlli
80005ec0   __divu
80002800   __divull
8000ad9c   __dtors_ptr
800069e0   __llshl
800076a0   __llshru
8000ada4   __lock
80007d00   __negll
80007d20   __nop
80007d40   __register_lock
80007d60   __register_unlock
80006580   __remu
8000bdb0   __stack
80006f60   __subcull
8000ada8   __unlock
80007d80   _abort
00000008   _argsize
80005f80   _atexit
80003d40   _c_int00
800054c0   _call_dtors
8000d7c8   _clk0
80004620   _clk0Fxn
8000d7cc   _clk1
80004644   _clk1Fxn
8000adac   _dtors
8000d7d8   _event0
800058c0   _exit
8000d7ec   _finishFlag
8000d7bc   _heap0
800045a4   _idl0Fxn
800076e0   _llabs
80004580   _main
8000d7e4   _mbx0
8000d7e8   _mbx1
80006620   _memcpy
800059a0   _memset
8000d7e0   _queue0
80006a60   _readmsg
8000d7d4   _sem0
8000d7dc   _sem1
8000d7c0   _swi0
800045d4   _swi0Fxn
8000d7c4   _swi1
800045f8   _swi1Fxn
8000468c   _task0Fxn
8000d7d0   _task1
800046b0   _task1Fxn
8000a450   _ti_sysbios_BIOS_Module__state__V
800066c0   _ti_sysbios_BIOS_exitFunc__I
80006ae0   _ti_sysbios_BIOS_exit__E
800017a0   _ti_sysbios_BIOS_startFunc__I
80007dc0   _ti_sysbios_BIOS_start__E
80007760   _ti_sysbios_family_c62_TaskSupport_buildTaskStack
80007de0   _ti_sysbios_family_c62_TaskSupport_glue
80006b60   _ti_sysbios_family_c62_TaskSupport_swap__E
8000a46c   _ti_sysbios_family_c64p_Cache_Module__state__V
80002a60   _ti_sysbios_family_c64p_Cache_Module_startup__E
80009a84   _ti_sysbios_family_c64p_Cache_initSize__C
80007e00   _ti_sysbios_family_c64p_Cache_setMar__E
8000a470   _ti_sysbios_family_c64p_Exception_Module__state__V
80007020   _ti_sysbios_family_c64p_Exception_Module_startup__E
80003bc0   _ti_sysbios_family_c64p_Exception_dispatch__E
80000ae0   _ti_sysbios_family_c64p_Exception_handler__I
8000d800   _ti_sysbios_family_c64p_Hwi0
8000d820   _ti_sysbios_family_c64p_Hwi1
8000d940   _ti_sysbios_family_c64p_Hwi10
8000d960   _ti_sysbios_family_c64p_Hwi11
8000d980   _ti_sysbios_family_c64p_Hwi12
8000d9a0   _ti_sysbios_family_c64p_Hwi13
8000d9c0   _ti_sysbios_family_c64p_Hwi14
8000d9e0   _ti_sysbios_family_c64p_Hwi15
8000d840   _ti_sysbios_family_c64p_Hwi2
8000d860   _ti_sysbios_family_c64p_Hwi3
8000d880   _ti_sysbios_family_c64p_Hwi4
8000d8a0   _ti_sysbios_family_c64p_Hwi5
8000d8c0   _ti_sysbios_family_c64p_Hwi6
8000d8e0   _ti_sysbios_family_c64p_Hwi7
8000d900   _ti_sysbios_family_c64p_Hwi8
8000d920   _ti_sysbios_family_c64p_Hwi9
8000a49c   _ti_sysbios_family_c64p_Hwi_Module__root__V
8000a4c0   _ti_sysbios_family_c64p_Hwi_Module__state__V
800046e0   _ti_sysbios_family_c64p_Hwi_Module_startup__E
8000a4a8   _ti_sysbios_family_c64p_Hwi_Object__table__V
80002ee0   _ti_sysbios_family_c64p_Hwi_dispatchAlways
80003ea0   _ti_sysbios_family_c64p_Hwi_dispatchC__I
80007e20   _ti_sysbios_family_c64p_TimestampProvider_Module_startup__E
80007e40   _ti_sysbios_family_c64p_ti81xx_TimerSupport_Module_startup__E
800077a0   _ti_sysbios_family_xxx_Hwi_switchToIsrStack
80007e60   _ti_sysbios_family_xxx_Hwi_switchToTaskStack
800077e0   _ti_sysbios_gates_GateHwi_Handle__label__S
80009880   _ti_sysbios_gates_GateHwi_Module__FXNS__C
8000a520   _ti_sysbios_gates_GateHwi_Module__root__V
80009910   _ti_sysbios_gates_GateHwi_Object__DESC__C
80009a10   _ti_sysbios_gates_GateHwi_Object__PARAMS__C
80007080   _ti_sysbios_gates_GateHwi_Object__create__S
80007820   _ti_sysbios_gates_GateHwi_Object__delete__S
8000a528   _ti_sysbios_gates_GateHwi_Object__table__V
80007e80   _ti_sysbios_gates_GateHwi_enter__E
80007ea0   _ti_sysbios_gates_GateHwi_leave__E
80007ec0   _ti_sysbios_gates_GateHwi_query__E
80007860   _ti_sysbios_gates_GateMutex_Handle__label__S
800078a0   _ti_sysbios_gates_GateMutex_Instance_finalize__F
800098a4   _ti_sysbios_gates_GateMutex_Module__FXNS__C
8000a52c   _ti_sysbios_gates_GateMutex_Module__root__V
80009930   _ti_sysbios_gates_GateMutex_Object__DESC__C
80009a28   _ti_sysbios_gates_GateMutex_Object__PARAMS__C
80006040   _ti_sysbios_gates_GateMutex_Object__create__S
800070e0   _ti_sysbios_gates_GateMutex_Object__delete__S
8000a538   _ti_sysbios_gates_GateMutex_Object__table__V
80005a80   _ti_sysbios_gates_GateMutex_enter__E
80007ee0   _ti_sysbios_gates_GateMutex_leave__E
80007f00   _ti_sysbios_gates_GateMutex_query__E
8000a558   _ti_sysbios_hal_Hwi_Module__root__V
800078e0   _ti_sysbios_hal_Hwi_Module_startup__E
8000a560   _ti_sysbios_hal_Hwi_Object__table__V
80006ee0   _ti_sysbios_hal_Hwi_checkStack
800075c0   _ti_sysbios_hal_Hwi_initStack
8000a568   _ti_sysbios_hal_Timer_Module__root__V
80007920   _ti_sysbios_hal_Timer_Module_startup__E
8000a570   _ti_sysbios_hal_Timer_Object__table__V
80007960   _ti_sysbios_heaps_HeapBuf_Handle__label__S
80009ab8   _ti_sysbios_heaps_HeapBuf_Instance_State_0_buf__A
800079a0   _ti_sysbios_heaps_HeapBuf_Instance_finalize__F
80001b00   _ti_sysbios_heaps_HeapBuf_Instance_init__F
80009830   _ti_sysbios_heaps_HeapBuf_Module__FXNS__C
8000a578   _ti_sysbios_heaps_HeapBuf_Module__root__V
8000a5a8   _ti_sysbios_heaps_HeapBuf_Module__state__V
80006100   _ti_sysbios_heaps_HeapBuf_Module_startup__E
80009950   _ti_sysbios_heaps_HeapBuf_Object__DESC__C
80009804   _ti_sysbios_heaps_HeapBuf_Object__PARAMS__C
800055c0   _ti_sysbios_heaps_HeapBuf_Object__create__S
80007140   _ti_sysbios_heaps_HeapBuf_Object__delete__S
8000a580   _ti_sysbios_heaps_HeapBuf_Object__table__V
800061c0   _ti_sysbios_heaps_HeapBuf_alloc__E
80006280   _ti_sysbios_heaps_HeapBuf_free__E
800071a0   _ti_sysbios_heaps_HeapBuf_getStats__E
80007f20   _ti_sysbios_heaps_HeapBuf_isBlocking__E
80006760   _ti_sysbios_knl_Clock_Instance_finalize__F
8000a5ac   _ti_sysbios_knl_Clock_Module__root__V
8000a5f8   _ti_sysbios_knl_Clock_Module__state__V
800079e0   _ti_sysbios_knl_Clock_Module_startup__E
80009970   _ti_sysbios_knl_Clock_Object__DESC__C
800098c8   _ti_sysbios_knl_Clock_Object__PARAMS__C
80004000   _ti_sysbios_knl_Clock_Object__create__S
8000a5b8   _ti_sysbios_knl_Clock_Object__table__V
80007200   _ti_sysbios_knl_Clock_doTick__I
80007a20   _ti_sysbios_knl_Clock_start__E
80004ce0   _ti_sysbios_knl_Clock_workFunc__E
8000a614   _ti_sysbios_knl_Event_Module__root__V
8000a620   _ti_sysbios_knl_Event_Object__table__V
80004160   _ti_sysbios_knl_Event_post__E
80009a90   _ti_sysbios_knl_Idle_funcList__A
80007a60   _ti_sysbios_knl_Idle_loop__E
80007260   _ti_sysbios_knl_Idle_run__E
80009bb8   _ti_sysbios_knl_Mailbox_Instance_State_0_allocBuf__A
80009bd8   _ti_sysbios_knl_Mailbox_Instance_State_1_allocBuf__A
8000a62c   _ti_sysbios_knl_Mailbox_Module__root__V
80005b60   _ti_sysbios_knl_Mailbox_Module_startup__E
8000a638   _ti_sysbios_knl_Mailbox_Object__table__V
8000a6e8   _ti_sysbios_knl_Queue_Module__root__V
80009990   _ti_sysbios_knl_Queue_Object__DESC__C
80009a40   _ti_sysbios_knl_Queue_Object__PARAMS__C
800072c0   _ti_sysbios_knl_Queue_Object__create__S
8000a6f0   _ti_sysbios_knl_Queue_Object__table__V
80007320   _ti_sysbios_knl_Semaphore_Instance_finalize__F
8000a6f8   _ti_sysbios_knl_Semaphore_Module__root__V
800099b0   _ti_sysbios_knl_Semaphore_Object__DESC__C
800098ec   _ti_sysbios_knl_Semaphore_Object__PARAMS__C
80004e00   _ti_sysbios_knl_Semaphore_Object__create__S
8000a700   _ti_sysbios_knl_Semaphore_Object__table__V
80006be0   _ti_sysbios_knl_Semaphore_pendTimeout__I
800013c0   _ti_sysbios_knl_Semaphore_pend__E
80004820   _ti_sysbios_knl_Semaphore_post__E
8000a7c8   _ti_sysbios_knl_Swi_Module_State_0_readyQ__A
8000a730   _ti_sysbios_knl_Swi_Module__root__V
8000a848   _ti_sysbios_knl_Swi_Module__state__V
80007f40   _ti_sysbios_knl_Swi_Module_startup__E
8000a738   _ti_sysbios_knl_Swi_Object__table__V
80006c60   _ti_sysbios_knl_Swi_post__E
80004f20   _ti_sysbios_knl_Swi_restoreHwi__E
80006340   _ti_sysbios_knl_Swi_run__I
800030e0   _ti_sysbios_knl_Swi_schedule__I
80009c38   _ti_sysbios_knl_Task_Instance_State_0_hookEnv__A
8000adb0   _ti_sysbios_knl_Task_Instance_State_0_stack__A
80009c40   _ti_sysbios_knl_Task_Instance_State_1_hookEnv__A
8000b1b0   _ti_sysbios_knl_Task_Instance_State_1_stack__A
80009c48   _ti_sysbios_knl_Task_Instance_State_2_hookEnv__A
8000b9b0   _ti_sysbios_knl_Task_Instance_State_2_stack__A
8000a940   _ti_sysbios_knl_Task_Module_State_0_readyQ__A
8000a864   _ti_sysbios_knl_Task_Module__root__V
8000a9c0   _ti_sysbios_knl_Task_Module__state__V
80002080   _ti_sysbios_knl_Task_Module_startup__E
8000a870   _ti_sysbios_knl_Task_Object__table__V
80007380   _ti_sysbios_knl_Task_allBlockedFunction__I
800036c0   _ti_sysbios_knl_Task_checkStacks__E
800073e0   _ti_sysbios_knl_Task_enter__I
800042c0   _ti_sysbios_knl_Task_exit__E
80009a58   _ti_sysbios_knl_Task_hooks__A
80004420   _ti_sysbios_knl_Task_schedule__I
80005040   _ti_sysbios_knl_Task_startup__E
80006ce0   _ti_sysbios_knl_Task_unblockI__E
8000aa50   _ti_sysbios_timers_dmtimer_Timer_Module_State_0_device__A
8000aa90   _ti_sysbios_timers_dmtimer_Timer_Module_State_0_handles__A
8000a9f4   _ti_sysbios_timers_dmtimer_Timer_Module__root__V
8000aaa4   _ti_sysbios_timers_dmtimer_Timer_Module__state__V
80006400   _ti_sysbios_timers_dmtimer_Timer_Module_startup__E
8000aa00   _ti_sysbios_timers_dmtimer_Timer_Object__table__V
80002cc0   _ti_sysbios_timers_dmtimer_Timer_setPeriodMicroSecs__E
800064c0   _ti_sysbios_timers_dmtimer_Timer_stop__E
80007aa0   _ti_sysbios_timers_dmtimer_Timer_stub__E
8000466c   _timer0Fxn
80007440   _writemsg
80006d60   _xdc_runtime_Assert_raise__I
80002300   _xdc_runtime_Core_createObject__I
80005c40   _xdc_runtime_Core_deleteObject__I
8000aab8   _xdc_runtime_Error_Module__state__V
800032e0   _xdc_runtime_Error_raiseX__E
800032e0   _xdc_runtime_Error_raiseX__F
80009a98   _xdc_runtime_IFilterLogger_Interface__BASE__C
80009a9c   _xdc_runtime_IGateProvider_Interface__BASE__C
80009aa0   _xdc_runtime_IHeap_Interface__BASE__C
80009aa4   _xdc_runtime_ILogger_Interface__BASE__C
80009aa8   _xdc_runtime_IModule_Interface__BASE__C
80007ae0   _xdc_runtime_LoggerBuf_Handle__label__S
80009c50   _xdc_runtime_LoggerBuf_Instance_State_0_entryArr__A
80007b20   _xdc_runtime_LoggerBuf_Instance_finalize__F
800097c8   _xdc_runtime_LoggerBuf_Module__FXNS__C
8000aabc   _xdc_runtime_LoggerBuf_Module__root__V
8000aaec   _xdc_runtime_LoggerBuf_Module__state__V
800074a0   _xdc_runtime_LoggerBuf_Module_startup__E
800099d0   _xdc_runtime_LoggerBuf_Object__DESC__C
80009858   _xdc_runtime_LoggerBuf_Object__PARAMS__C
80003a40   _xdc_runtime_LoggerBuf_Object__create__S
80007500   _xdc_runtime_LoggerBuf_Object__delete__S
8000aac8   _xdc_runtime_LoggerBuf_Object__table__V
80007f60   _xdc_runtime_LoggerBuf_disable__E
80007f80   _xdc_runtime_LoggerBuf_enable__E
80005160   _xdc_runtime_LoggerBuf_getFilterLevel__E
80005160   _xdc_runtime_LoggerBuf_getFilterLevel__F
80004960   _xdc_runtime_LoggerBuf_setFilterLevel__E
80004960   _xdc_runtime_LoggerBuf_setFilterLevel__F
80007b60   _xdc_runtime_LoggerBuf_write0__E
80007ba0   _xdc_runtime_LoggerBuf_write1__E
80007fa0   _xdc_runtime_LoggerBuf_write2__E
80006800   _xdc_runtime_LoggerBuf_write4__E
80006800   _xdc_runtime_LoggerBuf_write4__F
80005280   _xdc_runtime_LoggerBuf_write8__E
80005280   _xdc_runtime_LoggerBuf_write8__F
8000aaf4   _xdc_runtime_Memory_Module__state__V
800056c0   _xdc_runtime_Memory_alloc__F
80007be0   _xdc_runtime_Memory_free__E
8000aaf8   _xdc_runtime_Registry_Module__state__V
8000ab00   _xdc_runtime_Startup_Module__state__V
00000001   _xdc_runtime_Startup__EXECFXN__C
00000001   _xdc_runtime_Startup__RESETFXN__C
80007fc0   _xdc_runtime_Startup_exec__I
80009ab0   _xdc_runtime_Startup_firstFxns__A
800099f0   _xdc_runtime_Startup_sfxnRts__A
80009788   _xdc_runtime_Startup_sfxnTab__A
80003880   _xdc_runtime_Startup_startMods__I
8000a050   _xdc_runtime_SysMin_Module_State_0_outbuf__A
8000ab08   _xdc_runtime_SysMin_Module__state__V
80007c20   _xdc_runtime_SysMin_Module_startup__E
800053a0   _xdc_runtime_SysMin_flush__E
800053a0   _xdc_runtime_SysMin_flush__F
80007560   _xdc_runtime_SysMin_putch__E
80007560   _xdc_runtime_SysMin_putch__F
8000ab18   _xdc_runtime_System_Module_State_0_atexitHandlers__A
8000ab28   _xdc_runtime_System_Module__state__V
80007fe0   _xdc_runtime_System_Module_startup__E
800068a0   _xdc_runtime_System_abort__E
800068a0   _xdc_runtime_System_abort__F
80007c60   _xdc_runtime_System_aprintf__E
80000000   _xdc_runtime_System_doPrint__I
80008000   _xdc_runtime_System_exit__E
80008000   _xdc_runtime_System_exit__F
80001de0   _xdc_runtime_System_printfExtend__I
80007ca0   _xdc_runtime_System_printf__E
80006de0   _xdc_runtime_System_rtsExit__I
8000ab34   _xdc_runtime_Text_Module__state__V
80008040   _xdc_runtime_Text_charTab__A
80009610   _xdc_runtime_Text_nodeTab__A
80006e60   _xdc_runtime_Text_printVisFxn__I
800057c0   _xdc_runtime_Text_putMod__E
800057c0   _xdc_runtime_Text_putMod__F
80002580   _xdc_runtime_Text_putSite__E
80002580   _xdc_runtime_Text_putSite__F
80005d20   _xdc_runtime_Text_visitRope2__I
80008020   _xdc_runtime_Text_visitRope__I
80006940   _xdc_runtime_Text_xprintf__I
ffffffff   binit
8000cdb0   cinit
00001a74   const_size
80008040   const_start
ffffffff   edata
8000d7ee   end
ffffffff   etext
ffffffff   pinit


GLOBAL SYMBOLS: SORTED BY Symbol Address 

address    name
--------   ----
00000001   __TI_args_main
00000001   _xdc_runtime_Startup__EXECFXN__C
00000001   _xdc_runtime_Startup__RESETFXN__C
00000008   _argsize
00001000   __STACK_SIZE
00001a74   const_size
80000000   ___ASM__
80000000   _xdc_runtime_System_doPrint__I
80000060   ___ISA__
80000078   ___PLAT__
800000a0   ___TARG__
800000c0   ___TRDR__
80000ae0   _ti_sysbios_family_c64p_Exception_handler__I
800013c0   _ti_sysbios_knl_Semaphore_pend__E
800017a0   _ti_sysbios_BIOS_startFunc__I
80001b00   _ti_sysbios_heaps_HeapBuf_Instance_init__F
80001de0   _xdc_runtime_System_printfExtend__I
80002080   _ti_sysbios_knl_Task_Module_startup__E
80002300   _xdc_runtime_Core_createObject__I
80002580   _xdc_runtime_Text_putSite__E
80002580   _xdc_runtime_Text_putSite__F
80002800   __divull
80002a60   _ti_sysbios_family_c64p_Cache_Module_startup__E
80002cc0   _ti_sysbios_timers_dmtimer_Timer_setPeriodMicroSecs__E
80002ee0   _ti_sysbios_family_c64p_Hwi_dispatchAlways
800030e0   _ti_sysbios_knl_Swi_schedule__I
800032e0   _xdc_runtime_Error_raiseX__E
800032e0   _xdc_runtime_Error_raiseX__F
800036c0   _ti_sysbios_knl_Task_checkStacks__E
80003880   _xdc_runtime_Startup_startMods__I
80003a40   _xdc_runtime_LoggerBuf_Object__create__S
80003bc0   _ti_sysbios_family_c64p_Exception_dispatch__E
80003d40   _c_int00
80003ea0   _ti_sysbios_family_c64p_Hwi_dispatchC__I
80004000   _ti_sysbios_knl_Clock_Object__create__S
80004160   _ti_sysbios_knl_Event_post__E
800042c0   _ti_sysbios_knl_Task_exit__E
80004420   _ti_sysbios_knl_Task_schedule__I
80004580   _main
800045a4   _idl0Fxn
800045d4   _swi0Fxn
800045f8   _swi1Fxn
80004620   _clk0Fxn
80004644   _clk1Fxn
8000466c   _timer0Fxn
8000468c   _task0Fxn
800046b0   _task1Fxn
800046e0   _ti_sysbios_family_c64p_Hwi_Module_startup__E
80004820   _ti_sysbios_knl_Semaphore_post__E
80004960   _xdc_runtime_LoggerBuf_setFilterLevel__E
80004960   _xdc_runtime_LoggerBuf_setFilterLevel__F
80004aa0   __divlli
80004ce0   _ti_sysbios_knl_Clock_workFunc__E
80004e00   _ti_sysbios_knl_Semaphore_Object__create__S
80004f20   _ti_sysbios_knl_Swi_restoreHwi__E
80005040   _ti_sysbios_knl_Task_startup__E
80005160   _xdc_runtime_LoggerBuf_getFilterLevel__E
80005160   _xdc_runtime_LoggerBuf_getFilterLevel__F
80005280   _xdc_runtime_LoggerBuf_write8__E
80005280   _xdc_runtime_LoggerBuf_write8__F
800053a0   _xdc_runtime_SysMin_flush__E
800053a0   _xdc_runtime_SysMin_flush__F
800054c0   _call_dtors
800055c0   _ti_sysbios_heaps_HeapBuf_Object__create__S
800056c0   _xdc_runtime_Memory_alloc__F
800057c0   _xdc_runtime_Text_putMod__E
800057c0   _xdc_runtime_Text_putMod__F
800058c0   _exit
800059a0   _memset
80005a80   _ti_sysbios_gates_GateMutex_enter__E
80005b60   _ti_sysbios_knl_Mailbox_Module_startup__E
80005c40   _xdc_runtime_Core_deleteObject__I
80005d20   _xdc_runtime_Text_visitRope2__I
80005e00   _HOSTwrite
80005ec0   __c6xabi_divu
80005ec0   __divu
80005f80   _atexit
80006040   _ti_sysbios_gates_GateMutex_Object__create__S
80006100   _ti_sysbios_heaps_HeapBuf_Module_startup__E
800061c0   _ti_sysbios_heaps_HeapBuf_alloc__E
80006280   _ti_sysbios_heaps_HeapBuf_free__E
80006340   _ti_sysbios_knl_Swi_run__I
80006400   _ti_sysbios_timers_dmtimer_Timer_Module_startup__E
800064c0   _ti_sysbios_timers_dmtimer_Timer_stop__E
80006580   __c6xabi_remu
80006580   __remu
80006620   _memcpy
800066c0   _ti_sysbios_BIOS_exitFunc__I
80006760   _ti_sysbios_knl_Clock_Instance_finalize__F
80006800   _xdc_runtime_LoggerBuf_write4__E
80006800   _xdc_runtime_LoggerBuf_write4__F
800068a0   _xdc_runtime_System_abort__E
800068a0   _xdc_runtime_System_abort__F
80006940   _xdc_runtime_Text_xprintf__I
800069e0   __llshl
80006a60   _readmsg
80006ae0   _ti_sysbios_BIOS_exit__E
80006b60   _ti_sysbios_family_c62_TaskSupport_swap__E
80006be0   _ti_sysbios_knl_Semaphore_pendTimeout__I
80006c60   _ti_sysbios_knl_Swi_post__E
80006ce0   _ti_sysbios_knl_Task_unblockI__E
80006d60   _xdc_runtime_Assert_raise__I
80006de0   _xdc_runtime_System_rtsExit__I
80006e60   _xdc_runtime_Text_printVisFxn__I
80006ee0   _ti_sysbios_hal_Hwi_checkStack
80006f60   __subcull
80007020   _ti_sysbios_family_c64p_Exception_Module_startup__E
80007080   _ti_sysbios_gates_GateHwi_Object__create__S
800070e0   _ti_sysbios_gates_GateMutex_Object__delete__S
80007140   _ti_sysbios_heaps_HeapBuf_Object__delete__S
800071a0   _ti_sysbios_heaps_HeapBuf_getStats__E
80007200   _ti_sysbios_knl_Clock_doTick__I
80007260   _ti_sysbios_knl_Idle_run__E
800072c0   _ti_sysbios_knl_Queue_Object__create__S
80007320   _ti_sysbios_knl_Semaphore_Instance_finalize__F
80007380   _ti_sysbios_knl_Task_allBlockedFunction__I
800073e0   _ti_sysbios_knl_Task_enter__I
80007440   _writemsg
80007498   C$$IO$$
800074a0   _xdc_runtime_LoggerBuf_Module_startup__E
80007500   _xdc_runtime_LoggerBuf_Object__delete__S
80007560   _xdc_runtime_SysMin_putch__E
80007560   _xdc_runtime_SysMin_putch__F
800075c0   _ti_sysbios_hal_Hwi_initStack
80007620   ___add_dtor
80007660   __args_main
800076a0   __llshru
800076e0   _llabs
80007760   _ti_sysbios_family_c62_TaskSupport_buildTaskStack
800077a0   _ti_sysbios_family_xxx_Hwi_switchToIsrStack
800077e0   _ti_sysbios_gates_GateHwi_Handle__label__S
80007820   _ti_sysbios_gates_GateHwi_Object__delete__S
80007860   _ti_sysbios_gates_GateMutex_Handle__label__S
800078a0   _ti_sysbios_gates_GateMutex_Instance_finalize__F
800078e0   _ti_sysbios_hal_Hwi_Module_startup__E
80007920   _ti_sysbios_hal_Timer_Module_startup__E
80007960   _ti_sysbios_heaps_HeapBuf_Handle__label__S
800079a0   _ti_sysbios_heaps_HeapBuf_Instance_finalize__F
800079e0   _ti_sysbios_knl_Clock_Module_startup__E
80007a20   _ti_sysbios_knl_Clock_start__E
80007a60   _ti_sysbios_knl_Idle_loop__E
80007aa0   _ti_sysbios_timers_dmtimer_Timer_stub__E
80007ae0   _xdc_runtime_LoggerBuf_Handle__label__S
80007b20   _xdc_runtime_LoggerBuf_Instance_finalize__F
80007b60   _xdc_runtime_LoggerBuf_write0__E
80007ba0   _xdc_runtime_LoggerBuf_write1__E
80007be0   _xdc_runtime_Memory_free__E
80007c20   _xdc_runtime_SysMin_Module_startup__E
80007c60   _xdc_runtime_System_aprintf__E
80007ca0   _xdc_runtime_System_printf__E
80007ce0   ___xdc__init
80007d00   __negll
80007d20   __nop
80007d40   __register_lock
80007d60   __register_unlock
80007d80   C$$EXIT
80007d80   _abort
80007dc0   _ti_sysbios_BIOS_start__E
80007de0   _ti_sysbios_family_c62_TaskSupport_glue
80007e00   _ti_sysbios_family_c64p_Cache_setMar__E
80007e20   _ti_sysbios_family_c64p_TimestampProvider_Module_startup__E
80007e40   _ti_sysbios_family_c64p_ti81xx_TimerSupport_Module_startup__E
80007e60   _ti_sysbios_family_xxx_Hwi_switchToTaskStack
80007e80   _ti_sysbios_gates_GateHwi_enter__E
80007ea0   _ti_sysbios_gates_GateHwi_leave__E
80007ec0   _ti_sysbios_gates_GateHwi_query__E
80007ee0   _ti_sysbios_gates_GateMutex_leave__E
80007f00   _ti_sysbios_gates_GateMutex_query__E
80007f20   _ti_sysbios_heaps_HeapBuf_isBlocking__E
80007f40   _ti_sysbios_knl_Swi_Module_startup__E
80007f60   _xdc_runtime_LoggerBuf_disable__E
80007f80   _xdc_runtime_LoggerBuf_enable__E
80007fa0   _xdc_runtime_LoggerBuf_write2__E
80007fc0   _xdc_runtime_Startup_exec__I
80007fe0   _xdc_runtime_System_Module_startup__E
80008000   _xdc_runtime_System_exit__E
80008000   _xdc_runtime_System_exit__F
80008020   _xdc_runtime_Text_visitRope__I
80008040   _xdc_runtime_Text_charTab__A
80008040   const_start
80009610   _xdc_runtime_Text_nodeTab__A
80009788   _xdc_runtime_Startup_sfxnTab__A
800097c8   _xdc_runtime_LoggerBuf_Module__FXNS__C
80009804   _ti_sysbios_heaps_HeapBuf_Object__PARAMS__C
80009830   _ti_sysbios_heaps_HeapBuf_Module__FXNS__C
80009858   _xdc_runtime_LoggerBuf_Object__PARAMS__C
80009880   _ti_sysbios_gates_GateHwi_Module__FXNS__C
800098a4   _ti_sysbios_gates_GateMutex_Module__FXNS__C
800098c8   _ti_sysbios_knl_Clock_Object__PARAMS__C
800098ec   _ti_sysbios_knl_Semaphore_Object__PARAMS__C
80009910   _ti_sysbios_gates_GateHwi_Object__DESC__C
80009930   _ti_sysbios_gates_GateMutex_Object__DESC__C
80009950   _ti_sysbios_heaps_HeapBuf_Object__DESC__C
80009970   _ti_sysbios_knl_Clock_Object__DESC__C
80009990   _ti_sysbios_knl_Queue_Object__DESC__C
800099b0   _ti_sysbios_knl_Semaphore_Object__DESC__C
800099d0   _xdc_runtime_LoggerBuf_Object__DESC__C
800099f0   _xdc_runtime_Startup_sfxnRts__A
80009a10   _ti_sysbios_gates_GateHwi_Object__PARAMS__C
80009a28   _ti_sysbios_gates_GateMutex_Object__PARAMS__C
80009a40   _ti_sysbios_knl_Queue_Object__PARAMS__C
80009a58   _ti_sysbios_knl_Task_hooks__A
80009a84   _ti_sysbios_family_c64p_Cache_initSize__C
80009a90   _ti_sysbios_knl_Idle_funcList__A
80009a98   _xdc_runtime_IFilterLogger_Interface__BASE__C
80009a9c   _xdc_runtime_IGateProvider_Interface__BASE__C
80009aa0   _xdc_runtime_IHeap_Interface__BASE__C
80009aa4   _xdc_runtime_ILogger_Interface__BASE__C
80009aa8   _xdc_runtime_IModule_Interface__BASE__C
80009ab0   _xdc_runtime_Startup_firstFxns__A
80009ab8   _ti_sysbios_heaps_HeapBuf_Instance_State_0_buf__A
80009bb8   _ti_sysbios_knl_Mailbox_Instance_State_0_allocBuf__A
80009bd8   _ti_sysbios_knl_Mailbox_Instance_State_1_allocBuf__A
80009c38   _ti_sysbios_knl_Task_Instance_State_0_hookEnv__A
80009c40   _ti_sysbios_knl_Task_Instance_State_1_hookEnv__A
80009c48   _ti_sysbios_knl_Task_Instance_State_2_hookEnv__A
80009c50   _xdc_runtime_LoggerBuf_Instance_State_0_entryArr__A
8000a050   _xdc_runtime_SysMin_Module_State_0_outbuf__A
8000a450   _ti_sysbios_BIOS_Module__state__V
8000a46c   _ti_sysbios_family_c64p_Cache_Module__state__V
8000a470   _ti_sysbios_family_c64p_Exception_Module__state__V
8000a49c   _ti_sysbios_family_c64p_Hwi_Module__root__V
8000a4a8   _ti_sysbios_family_c64p_Hwi_Object__table__V
8000a4c0   _ti_sysbios_family_c64p_Hwi_Module__state__V
8000a520   _ti_sysbios_gates_GateHwi_Module__root__V
8000a528   _ti_sysbios_gates_GateHwi_Object__table__V
8000a52c   _ti_sysbios_gates_GateMutex_Module__root__V
8000a538   _ti_sysbios_gates_GateMutex_Object__table__V
8000a558   _ti_sysbios_hal_Hwi_Module__root__V
8000a560   _ti_sysbios_hal_Hwi_Object__table__V
8000a568   _ti_sysbios_hal_Timer_Module__root__V
8000a570   _ti_sysbios_hal_Timer_Object__table__V
8000a578   _ti_sysbios_heaps_HeapBuf_Module__root__V
8000a580   _ti_sysbios_heaps_HeapBuf_Object__table__V
8000a5a8   _ti_sysbios_heaps_HeapBuf_Module__state__V
8000a5ac   _ti_sysbios_knl_Clock_Module__root__V
8000a5b8   _ti_sysbios_knl_Clock_Object__table__V
8000a5f8   _ti_sysbios_knl_Clock_Module__state__V
8000a614   _ti_sysbios_knl_Event_Module__root__V
8000a620   _ti_sysbios_knl_Event_Object__table__V
8000a62c   _ti_sysbios_knl_Mailbox_Module__root__V
8000a638   _ti_sysbios_knl_Mailbox_Object__table__V
8000a6e8   _ti_sysbios_knl_Queue_Module__root__V
8000a6f0   _ti_sysbios_knl_Queue_Object__table__V
8000a6f8   _ti_sysbios_knl_Semaphore_Module__root__V
8000a700   _ti_sysbios_knl_Semaphore_Object__table__V
8000a730   _ti_sysbios_knl_Swi_Module__root__V
8000a738   _ti_sysbios_knl_Swi_Object__table__V
8000a7c8   _ti_sysbios_knl_Swi_Module_State_0_readyQ__A
8000a848   _ti_sysbios_knl_Swi_Module__state__V
8000a864   _ti_sysbios_knl_Task_Module__root__V
8000a870   _ti_sysbios_knl_Task_Object__table__V
8000a8f8   _TSK_idle
8000a940   _ti_sysbios_knl_Task_Module_State_0_readyQ__A
8000a9c0   _ti_sysbios_knl_Task_Module__state__V
8000a9f4   _ti_sysbios_timers_dmtimer_Timer_Module__root__V
8000aa00   _ti_sysbios_timers_dmtimer_Timer_Object__table__V
8000aa50   _ti_sysbios_timers_dmtimer_Timer_Module_State_0_device__A
8000aa90   _ti_sysbios_timers_dmtimer_Timer_Module_State_0_handles__A
8000aaa4   _ti_sysbios_timers_dmtimer_Timer_Module__state__V
8000aab8   _xdc_runtime_Error_Module__state__V
8000aabc   _xdc_runtime_LoggerBuf_Module__root__V
8000aac8   _xdc_runtime_LoggerBuf_Object__table__V
8000aaec   _xdc_runtime_LoggerBuf_Module__state__V
8000aaf4   _xdc_runtime_Memory_Module__state__V
8000aaf8   _xdc_runtime_Registry_Module__state__V
8000ab00   _xdc_runtime_Startup_Module__state__V
8000ab08   _xdc_runtime_SysMin_Module__state__V
8000ab18   _xdc_runtime_System_Module_State_0_atexitHandlers__A
8000ab28   _xdc_runtime_System_Module__state__V
8000ab34   _xdc_runtime_Text_Module__state__V
8000ab3c   ___xdc__init__addr
8000ab40   ___atexit_func_id__
8000ad98   __cleanup_ptr
8000ad9c   __dtors_ptr
8000ada0   ___TI_enable_exit_profile_output
8000ada4   __lock
8000ada8   __unlock
8000adac   _dtors
8000adb0   _ti_sysbios_knl_Task_Instance_State_0_stack__A
8000b1b0   _ti_sysbios_knl_Task_Instance_State_1_stack__A
8000b9b0   _ti_sysbios_knl_Task_Instance_State_2_stack__A
8000bdb0   __stack
8000cdb0   __STACK_END
8000cdb0   ___cinit__
8000cdb0   cinit
8000d7bc   $bss
8000d7bc   .bss
8000d7bc   ___bss__
8000d7bc   _heap0
8000d7c0   _swi0
8000d7c4   _swi1
8000d7c8   _clk0
8000d7cc   _clk1
8000d7d0   _task1
8000d7d4   _sem0
8000d7d8   _event0
8000d7dc   _sem1
8000d7e0   _queue0
8000d7e4   _mbx0
8000d7e8   _mbx1
8000d7ec   _finishFlag
8000d7ee   ___end__
8000d7ee   end
8000d7f0   ___c_args__
8000d800   _ti_sysbios_family_c64p_Hwi0
8000d820   _ti_sysbios_family_c64p_Hwi1
8000d840   _ti_sysbios_family_c64p_Hwi2
8000d860   _ti_sysbios_family_c64p_Hwi3
8000d880   _ti_sysbios_family_c64p_Hwi4
8000d8a0   _ti_sysbios_family_c64p_Hwi5
8000d8c0   _ti_sysbios_family_c64p_Hwi6
8000d8e0   _ti_sysbios_family_c64p_Hwi7
8000d900   _ti_sysbios_family_c64p_Hwi8
8000d920   _ti_sysbios_family_c64p_Hwi9
8000d940   _ti_sysbios_family_c64p_Hwi10
8000d960   _ti_sysbios_family_c64p_Hwi11
8000d980   _ti_sysbios_family_c64p_Hwi12
8000d9a0   _ti_sysbios_family_c64p_Hwi13
8000d9c0   _ti_sysbios_family_c64p_Hwi14
8000d9e0   _ti_sysbios_family_c64p_Hwi15
8000da00   __CIOBUF_
ffffffff   .data
ffffffff   .text
ffffffff   ___TI_pprof_out_hndl
ffffffff   ___TI_prof_data_size
ffffffff   ___TI_prof_data_start
ffffffff   ___binit__
ffffffff   ___data__
ffffffff   ___edata__
ffffffff   ___etext__
ffffffff   ___pinit__
ffffffff   ___text__
ffffffff   binit
ffffffff   edata
ffffffff   etext
ffffffff   pinit

[337 symbols]
